:020000040800F2
:1000000000070020E5040008B91D0008391D00089C
:10001000911D0008391D0008651D0008E70400084F
:10002000E7040008E7040008E7040008B1450008F9
:10003000E7040008E7040008E7040008E7040008F4
:10004000E7040008E7040008E7040008E7040008E4
:10005000E7040008E70400084D5600087956000838
:10006000A5560008D1560008FD560008E704000810
:10007000E7040008E7040008E7040008E7040008B4
:10008000E7040008E7040008E7040008712D0008F1
:10009000DD2D0008312E0008852E000829570008A4
:1000A000E7040008E7040008E7040008E704000884
:1000B000C1540008E7040008E7040008E70400084A
:1000C000E7040008E7040008E7040008E704000864
:1000D000E7040008E7040008E7040008E704000854
:1000E00091570008E7040008E7040008E704000847
:1000F000E7040008E7040008E7040008E704000834
:10010000E7040008E7040008E7040008E704000823
:10011000E7040008E7040008E7040008E704000813
:10012000E7040008E7040008E7040008E704000803
:10013000E7040008E7040008E7040008E7040008F3
:10014000E7040008E7040008E7040008E94C000899
:10015000E7040008E7040008E7040008E7040008D3
:10016000E7040008E7040008E7040008E7040008C3
:10017000E7040008E7040008E7040008E7040008B3
:10018000E7040008E7040008E7040008E7040008A3
:10019000E7040008E7040008E7040008E704000893
:1001A000E7040008E7040008E7040008E704000883
:1001B000E7040008E7040008E7040008E704000873
:1001C000E7040008E7040008E7040008E704000863
:1001D000E7040008E7040008E7040008E704000853
:1001E00053B94AB9002908BF00281CBF4FF0FF319E
:1001F0004FF0FF3000F074B9ADF1080C6DE904CE9A
:1002000000F006F8DDF804E0DDE9022304B07047F1
:100210002DE9F047089D04468E46002B4DD18A42B9
:10022000944669D9B2FA82F252B101FA02F3C2F1EC
:10023000200120FA01F10CFA02FC41EA030E94407D
:100240004FEA1C48210CBEFBF8F61FFA8CF708FB9E
:1002500016E341EA034306FB07F199420AD91CEB76
:10026000030306F1FF3080F01F81994240F21C81A8
:10027000023E63445B1AA4B2B3FBF8F008FB1033F0
:1002800044EA034400FB07F7A7420AD91CEB040425
:1002900000F1FF3380F00A81A74240F207816444F5
:1002A000023840EA0640E41B00261DB1D44000237A
:1002B000C5E900433146BDE8F0878B4209D9002DDE
:1002C00000F0EF800026C5E9000130463146BDE868
:1002D000F087B3FA83F6002E4AD18B4202D38242D2
:1002E00000F2F980841A61EB030301209E46002D81
:1002F000E0D0C5E9004EDDE702B9FFDEB2FA82F2D6
:10030000002A40F09280A1EB0C014FEA1C471FFA33
:100310008CFE0126200CB1FBF7F307FB131140EA1A
:1003200001410EFB03F0884208D91CEB010103F1E7
:10033000FF3802D2884200F2CB804346091AA4B2A9
:10034000B1FBF7F007FB101144EA01440EFB00FE7D
:10035000A64508D91CEB040400F1FF3102D2A645E2
:1003600000F2BB800846A4EB0E0440EA03409CE781
:10037000C6F12007B34022FA07FC4CEA030C20FA2E
:1003800007F401FA06F31C43F9404FEA1C4900FA4E
:1003900006F3B1FBF9F8200C1FFA8CFE09FB1811CB
:1003A00040EA014108FB0EF0884202FA06F20BD93E
:1003B0001CEB010108F1FF3A80F08880884240F28E
:1003C0008580A8F102086144091AA4B2B1FBF9F0D2
:1003D00009FB101144EA014100FB0EFE8E4508D9CD
:1003E0001CEB010100F1FF346CD28E456AD9023852
:1003F000614440EA0840A0FB0294A1EB0E01A14237
:10040000C846A64656D353D05DB1B3EB080261EBA4
:100410000E0101FA07F722FA06F3F1401F43C5E97E
:10042000007100263146BDE8F087C2F12003D840B4
:100430000CFA02FC21FA03F3914001434FEA1C47F6
:100440001FFA8CFEB3FBF7F007FB10360B0C43EAE8
:10045000064300FB0EF69E4204FA02F408D91CEB98
:10046000030300F1FF382FD29E422DD90238634496
:100470009B1B89B2B3FBF7F607FB163341EA034136
:1004800006FB0EF38B4208D91CEB010106F1FF3885
:1004900016D28B4214D9023E6144C91A46EA00467C
:1004A00038E72E46284605E70646E3E61846F8E60E
:1004B0004B45A9D2B9EB020864EB0C0E0138A3E757
:1004C0004646EAE7204694E74046D1E7D0467BE738
:1004D000023B614432E7304609E76444023842E7B0
:1004E000704700BF02E000F000F8FEE772B63A483D
:1004F00080F30888394880F3098839484EF6085156
:10050000CEF20001086040F20000CCF200004EF68E
:100510003471CEF200010860BFF34F8FBFF36F8FCD
:1005200040F20000C0F2F0004EF68851CEF2000119
:100530000860BFF34F8FBFF36F8F4FF00000E1EE05
:10054000100A4EF63C71CEF200010860062080F3DE
:100550001488BFF36F8F04F0ABF804F087F804F051
:1005600013FF4FF055301F491B4A91423CBF41F8E1
:10057000040BFAE71C49194A91423CBF41F8040BAD
:10058000FAE71A491A4A1B4B9A423EBF51F8040B2C
:1005900042F8040BF8E700201749184A91423CBF83
:1005A00041F8040BFAE704F065F804F041FF144C3D
:1005B000144DAC4203DA54F8041B8847F9E700F005
:1005C00041F8114C114DAC4203DA54F8041B884732
:1005D000F9E704F04DB800000007002000230020D8
:1005E000000000080001002000070020E05C000877
:1005F00000230020542300205823002028400020FE
:10060000E0010008E0010008E0010008E001000846
:100610002DE9F04F2DED108AC1F80CD0C3689D462E
:10062000BDEC108ABDE8F08F002383F311882846C3
:10063000A047002003F046FBFEE703F0C1FA00DF0D
:10064000FEE70000F8B503F051FF074603F09CFFFA
:100650000546A0BB1F4B9F4231D001339F4231D092
:100660001D4B27F0FF029A422FD1F8B200F022FD75
:100670002E4642F2107400F027FF08B100242646EF
:1006800000F01EFD08B90646044635B1134B9F42E3
:1006900003D003F071FF00242646002003F030FF52
:1006A0000EB100F063F801F019FB00F06BFF01F0F0
:1006B000A5F9204600F0B6F800F058F8F9E72E4604
:1006C0000024D8E704460126D5E7064641F28834DF
:1006D000D1E700BF010007B0000008B0263A09B01A
:1006E00008B501F05DF9A0F120035842584108BD5A
:1006F00007B541F21203022101A8ADF8043001F060
:100700006DF903B05DF804FB10B5202383F3118865
:100710001248C3680BB103F05BFB114A0F4800237A
:100720004FF47A7103F018FB002383F311880D4C0A
:10073000236813B12368013B2360636813B16368C6
:10074000013B6360084B1B7833B9636823B902200F
:1007500001F03EFA3223636010BD00BF5823002031
:1007600009070008742400206C230020274B284A26
:1007700010B51C461968013146D004339342F9D1B3
:100780006268244B9A423FD9234B9B6803F1006374
:1007900003F580339A4237D203F0C2FE03F0D4FE51
:1007A000002001F045F91D4B0220187001F006FAF7
:1007B0001B4B1A6C00221A64196E1A66196E596C5A
:1007C0005A64596E5A665A6E5A6942F080025A61EA
:1007D0005A6922F080025A615A691A6942F000523D
:1007E0001A611A6922F000521A611B6972B64FF041
:1007F000E0232021C3F8084DD4E9003281F31188A9
:100800009D4683F30888104710BD00BF0000010813
:1008100020000108FFFF0008002300206C230020B7
:10082000003802402DE9F04F93B0AC4B00902022ED
:10083000FF210AA89D6801F0FBF9A94A1378A3B922
:10084000A8480121C3601170202383F31188C36875
:100850000BB103F0BDFAA44AA24800234FF47A7109
:1008600003F07AFA002383F31188009B9F4A03B1B7
:1008700013609F49009C00230B70536098469B4671
:100880001E469A46012001F099F924B1974B1B6846
:10089000002B00F01C82002001F082F80390039BE3
:1008A000002B01DA00F020FF039B002BEDDB012081
:1008B00001F07AF9039B213B162BE3D801A252F8F1
:1008C00023F000BF2109000849090008DD090008DC
:1008D000850800088508000885080008710A0008D6
:1008E000430C00085D0B0008BF0B0008E70B000875
:1008F0000D0C0008850800081F0C0008850800087A
:10090000910C0008C109000885080008D50C0008F2
:100910002D090008C109000885080008BF0B000860
:100920000220FFF7DDFE002840F0FB81009B022142
:10093000B8F1000F08BF1C4605A841F21233ADF80C
:10094000143001F04BF89DE74FF47A7001F028F86D
:10095000071EEBDB0220FFF7C3FE0028E6D0013FB5
:10096000052F00F2E081DFE807F0030A0D101336CF
:1009700005230593042105A801F030F817E0574836
:100980000421F9E75B480421F6E75B480421F3E71B
:100990004FF01C09484601F04DF809F10409059093
:1009A000042105A801F01AF8B9F12C0FF2D10120A9
:1009B00000FA07F747EA0B0B5FFA8BFB4FF0000AD0
:1009C00001F082F926B10BF00B030B2B08BF0024BA
:1009D000FFF78EFE56E749480421CDE7002EA5D04B
:1009E0000BF00B030B2BA1D10220FFF779FE07467A
:1009F00000289BD001203E4E01F01AF802203070F2
:100A000001F0DCF84FF000085FFA88F9484601F081
:100A10001FF8044690B1484601F02AF808F1010891
:100A20000028F1D1B846044641F21213022105A86C
:100A3000ADF814303E4600F0D1FF23E70123022039
:100A4000337001F0B1F82546244B9B68AB4207D9BF
:100A5000284600F0EFFF013040F068810435F3E7ED
:100A6000234B00251D70214BB8465D603E46A7E72D
:100A7000002E3FF45BAF0BF00B030B2B7FF456AF54
:100A80001B4B0220187001F099F8322000F088FF0B
:100A9000B0F10009FFF64AAF19F003077FF446AF43
:100AA0000E4A926809EB050393423FF63FAFB9F552
:100AB000807F3FF73BAF124B0193B94522DD4FF4E6
:100AC0007A7000F06DFF0390039A002AFFF62EAFB4
:100AD000019B039A03F8012B0137EDE70023002067
:100AE00070240020582300200907000874240020E7
:100AF0006C23002004230020082300200C23002066
:100B000070230020C820FFF7EBFD074600283FF4C4
:100B10000DAF1F2D11D8C5F120024A450AAB25F0B3
:100B2000030028BF4A4683490192184401F05AF84D
:100B3000019A8048FF2101F07BF84FEAA9037D4923
:100B40000193C9F38702284601F07AF80646002887
:100B50003FF46AAF019B05EB830531E70220FFF705
:100B6000BFFD00283FF4E2AE00F0ACFF00283FF4E8
:100B7000DDAE0027B946704B9B68BB4218D91F2FCA
:100B800011D80A9B01330ED027F0030312AA134495
:100B900053F8203C05934846042205A901F012F9B8
:100BA00004378146E7E7384600F044FF0590F2E756
:100BB000CDF81490042105A800F010FF00E70023F1
:100BC000642104A8049300F0FFFE00287FF4AEAE79
:100BD0000220FFF785FD00283FF4A8AE049800F03E
:100BE00059FF0590E6E70023642104A8049300F070
:100BF000EBFE00287FF49AAE0220FFF771FD00287B
:100C00003FF494AE049800F055FFEAE70220FFF7A6
:100C100067FD00283FF48AAE00F064FFE1E70220A0
:100C2000FFF75EFD00283FF481AE05A9142000F017
:100C30005FFF04210746049004A800F0CFFE394668
:100C4000B9E7322000F0ACFE071EFFF66FAEBB071F
:100C50007FF46CAE384A926807EB0A0393423FF682
:100C600065AE0220FFF73CFD00283FF45FAE27F0A1
:100C700003075744BA453FF4A3AE504600F0DAFEEE
:100C80000421059005A800F0A9FE0AF1040AF1E785
:100C90004FF47A70FFF724FD00283FF447AE00F0D0
:100CA00011FF002844D00A9B01330BD008220AA967
:100CB000002000F0C5FF00283AD02022FF210AA81A
:100CC00000F0B6FFFFF714FD1C4803F001F813B065
:100CD000BDE8F08F002E3FF429AE0BF00B030B2B79
:100CE0007FF424AE0023642105A8059300F06CFE78
:100CF000074600287FF41AAE0220FFF7F1FC814678
:100D000000283FF413AEFFF7F3FC41F2883002F005
:100D1000DFFF059801F00AF84E4600F0D5FF3C468B
:100D2000B0E506464CE64FF0000AFFE5B8467BE624
:100D3000374679E67023002000230020A0860100BA
:100D4000094A136849F2690099B21B0C00FB013390
:100D50001360064B186844F2506182B2000C01FB2C
:100D60000200186080B27047202300201C2300205E
:100D700010B500211022044600F05AFF034B03CBAC
:100D8000206061601868A06010BD00BF107AFF1F6E
:100D90002DE9F043224DBBB001F010F8AB6840F2F2
:100DA000ED22C31A934232D906AFA8602B462822FF
:100DB0000021384601F010FD05F10E0000F030FF73
:100DC000002604465FFA80F905F10E08F3B2F1003F
:100DD000994501F1280107D908EB06030822384696
:100DE00001F0FAFC0136F1E708230122CDE90232D5
:100DF00005340C4B0193A4B230230093CDE9047465
:100E000005A3D3E90023297B074801F0FDFA3BB095
:100E1000BDE8F083AFF3008078F6339F93CACD8DA1
:100E2000C0340020CD3400209434002070B50D462D
:100E300014461E4601F07EFA50B9022E10D1012C44
:100E40000ED112A3D3E90023C5E90023012007E056
:100E5000282C10D005D8012C09D0052C0FD000204B
:100E600070BD302CFBD10BA3D3E90023ECE70BA31F
:100E7000D3E90023E8E70BA3D3E90023E4E70BA3BE
:100E8000D3E90023E0E700BFAFF30080401DA120BD
:100E900026812A0B78F6339F93CACD8D9E6AC42192
:100EA000818A46EE26417272DF25D7B7F017304AA5
:100EB00039059E5613B504462346084620220021D4
:100EC000019001F089FC22790198032A234628BF6A
:100ED000032203F8042F2021022201F07DFC627915
:100EE0000198072A234628BF072203F8052F22214D
:100EF000032201F071FCA2790198072A234628BF3A
:100F0000072203F8062F2521032201F065FC019832
:100F100004F108031022282101F05EFC382002B001
:100F200010BD00002DE9F04FADF5017D21AD0EAEF5
:100F300040F2751280460F4622A80021296000F079
:100F400077FE48220021304600F072FE00F036FFA6
:100F5000564B4FF47A72B0FBF2F0186093E807003A
:100F6000012386E807000DF15A003382FFF700FFE6
:100F70004FF20363338407AB18464D4904F0B4FCC9
:100F80001B2230642946304686F83C20FFF792FF4A
:100F900012AB044601460822284601F01DFC082237
:100FA000A1180DF14903284601F016FC0DF14A0382
:100FB000082204F11001284601F00EFC13AB202298
:100FC00004F11801284601F007FC14AB402204F19B
:100FD0003801284601F000FC16AB082204F1780124
:100FE000284601F0F9FB0DF15903082204F18001B4
:100FF000284601F0F1FB04F1880A0DF15A0904F5C5
:10100000847B4B465146082228460AF1080A01F023
:10101000E3FBD34509F10109F3D11BAB0822594683
:10102000284601F0D9FB04F588744FF0000996F8C2
:1010300034304B450AD9B36B21464B44082228462D
:1010400001F0CAFB083409F10109F0E74FF000098B
:1010500096F83C304B4504EBC90108D9336C0822A3
:101060004B44284601F0B8FB09F10109F0E70023E1
:101070000393BB7E0293073107F119030193C1F378
:10108000CF010123CDE904510093F97E05A3D3E9F3
:101090000023404601F0B8F90DF5017DBDE8F08F61
:1010A000AFF300809E6AC421818A46EE7C24002032
:1010B000F8580008014B1870704700BF88240020C2
:1010C000F0B5334B1C7B85B034B1324B0E221A8104
:1010D0000024204605B0F0BD2F4A1068516802ABCD
:1010E00003C308232D492E480DEB030204F0DAFB5D
:1010F000054630B9274B2B480A221A8100F018FE0A
:10110000E6E70169B1F5702F06D9224B26480B227C
:101110001A8100F00DFEDCE7438B40F2F632934279
:1011200007D01C490C2008811946204800F000FE19
:10113000CFE71F4A024402F11003994204D2154B33
:101140001C4810221A81E4E710398E1A20461449EF
:1011500000F038FE3246074605F11801204600F03F
:1011600031FEAB689F4202D1EB6898420AD0094B2E
:101170000D221A810090D5E902123B460E4800F07C
:10118000D7FDA5E70D4800F0D3FD0124A1E700BF7E
:10119000C03400207C240020A5590008DCFF0E008C
:1011A00000000108145900082059000832590008AD
:1011B0000800FFF7505900086D59000896590008BB
:1011C0002DE9F04FADB006AF80460C4601F0B2F805
:1011D000054600285AD1237E022B1BD1E38A012B1E
:1011E00018D100F0EBFD0646FFF7AAFD03464FF4C9
:1011F000C870DFF8D092B3FBF0F206F5167602FB6A
:10120000103316FA83F3C9F80030E37E33B9A84BE4
:1012100000221A709C37BD46BDE8F08FA38AEEB25B
:10122000013BB34205F101050BD93B1D1E44E9000A
:1012300000960023082201F0F801204601F090F901
:10124000ECE707F11400FFF793FD324607F11401B4
:10125000381D04F017FB0028D9D10F2E08D8944B65
:101260001E70D9F80030A3F51673C9F80030D1E725
:10127000FB1CF8700146009307220346204601F04C
:101280006FF9F978404601F04DF8C3E7E38A282B5F
:1012900026D010D8012B1ED0052BBBD1BFF34F8F0A
:1012A0008449854BCA6802F4E0621343CB60BFF304
:1012B0004F8F00BFFDE7302BACD1637E7F4D0133F4
:1012C0006A7BDBB29342E94603D1E27E2B7B9A42F2
:1012D00065D0CD469EE721464046FFF723FE99E7BD
:1012E000A38A013B9BB2C92B94D8744D2E7B26BB9D
:1012F00005F10C030093082233463146204601F0E5
:101300002FF9731CF2B2D9001E46A38A013B9A4200
:1013100005DA0E322A44009200230822EEE7002369
:101320000022C5E900230023AB6085F8D730C5F85B
:10133000D8302B7B0BB9E37E2B73002507F1140902
:101340003B1D082229464846C7E90155FD6001F0CA
:1013500043FA3B7A05F1010AAB424FEACA0608D9C3
:10136000FB6808222B443146484601F035FA5546C1
:10137000EFE7C6F3CF06E17ECDE9049600230393A1
:10138000A37E0293193428230093019446A3D3E942
:101390000023404601F038F8FFF7FAFC3AE74FF037
:1013A000000807F11403A7F81480102200934146A7
:1013B0000123204601F0D4F8A68A023EB6B2F31CFF
:1013C0009B109B000733DB08A9EBC3039D460DF17F
:1013D000180A1FFA88F34FEAC801B34201F110015D
:1013E0000AD20AEB0803009308220023204601F0EA
:1013F000B7F808F10108ECE795F8D70000F028FBF2
:10140000D5F8D83004461BB995F8D70000F030FB6A
:10141000D5F8D83033449C4204D295F8D700013037
:1014200000F026FB4FEA960B4FF000081FFA88F1F8
:101430008B45D5E9003209D90AEB880103EB880016
:10144000012200F0FDFB08F10108EFE7F31842F17B
:101450000002C5E90032D5F8D83095F8D70006EB80
:101460000308C5F8D88000F0F3FA804509D395F851
:10147000D730D5F8D8000133001B85F8D730C5F830
:10148000D800FF2E08D800232B7300F01BFBFFF7BA
:1014900017FE08B1FFF76AF92B68094A9B0A013366
:1014A00013810023AB6014E726417272DF25D7B7A2
:1014B0008D34002000ED00E00400FA05C034002067
:1014C0007C2400209034002030B54FF00054244B91
:1014D00022689A4285B007D003F060F80446A8B9A4
:1014E0000024204605B030BD1E4B627D1A701E4898
:1014F000237D03731D49C9220E3000F073FB204683
:10150000E022002100F094FB0124EAE7184A194D7B
:10151000136C43F000731364AA6D174B9A42DFD12A
:101520002B6E013B7E2BDBD8144A07CA01AB83E844
:1015300007001846032100F05BFC6B6D83424FF0FF
:101540000003CDD12A6D8A4201BFAB65054B2A6EDF
:101550001A7003BF0A4BEA6D1A601C46C1E700BF50
:101560009AAD44C588240020C03400201600002015
:1015700000380240006600405041A0B0586600406C
:10158000182300202DE9FF474B4C022363710023F1
:1015900002934A4BD3F800C0BCF57A7F12D3484B74
:1015A000484FB7FBFCF69C458CBF0A231123581EFD
:1015B000B6FBF3F503FB1562C1B2002A3ED0022848
:1015C0000346F4D89DF80B303F4940485A1E9DF819
:1015D0000A30013B1B0443EA0253BDF80820013ADC
:1015E00013434B6001F0B0FD00230193384B3949A0
:1015F00000933948394B4FF4805200F06DFE384B60
:10160000197811B1344800F08DFE00F0D7FB054683
:10161000FFF796FB4FF4C873B0FBF3F202FB130322
:1016200005F5167010FA83F02E4B186002F0ACFF2F
:1016300008B10F23238104B0BDE8F0876B1EB3F51A
:10164000806FBFD2C1EBC10E0EF103034FEAE30975
:10165000C3F3C703A1EB030809F1010A4FF47A7041
:101660005FFA88F609FB00005AFA88F8B0FBF8F038
:10167000B0F5617F08D90EF1FF33C3F3C703C91A70
:10168000CEB2591E0F2914D8721E072A8CBF002211
:101690000122991901FB0551B7FBF1F7BC4591D126
:1016A000002A8FD0ADF808508DF80A308DF80B6005
:1016B00088E71346EDE700BF7C24002018230020B4
:1016C0003F420F0080DE800210230020D83500202A
:1016D0002D0E00088C24002094340020C111000835
:1016E00088240020903400202DE9F04F91A7D7E9FD
:1016F00000670FF24829D9E90089874D93B0DFF8D8
:1017000044B2864C284600F0E3FE0DF1300A079003
:1017100070B310220021504600F08AFA079B197B13
:101720004FF0000261F303028DF830205868996889
:101730000EAA03C21B680D9A63F31C029DF8303099
:101740000D9243F020038DF83030002352461946A5
:10175000584601F009FD079028B9284600F0BCFE64
:10176000079B2370CEE72378072B3CD801332370E7
:1017700018220021504600F05BFADFF8C8B1684C2F
:10178000002319465246584601F016FD014670BB2B
:10179000102208A800F04CFA636983F48043636167
:1017A00000F00EFB0B4612A9024611E903000DF1F1
:1017B000240C8CE803009DF83410C1F30300890663
:1017C0004CBF0E99BDF838C08DF82C0046BFC1F350
:1017D0001C0C4CF00041CCF30A010891284608A9E2
:1017E00001F042F8CCE7284600F076FEC0E7284634
:1017F00000F0A0FD0446002848D1DFF84CB100F00D
:10180000DDFADBF80030984240D300F0D7FA0790B9
:10181000FFF796FA079A8DF8204003464FF4C870F8
:1018200002F51672B3FBF0F101FB103312FA83F3E9
:10183000CBF80030DFF814B19BF8001011B9012388
:101840008DF8203050460791FFF792FA0799C1F1C1
:101850001004E4B2062C28BF0624224651440DF1A0
:10186000210000F0BFF908AB039318230293013461
:101870002C4B0193E4B20123009304943B4632467F
:10188000284600F059FD00238BF8003000F096FA4E
:10189000254A264C1368C31AB3F57A7F31D31060FA
:1018A00000F08EFA02460B46284600F01FFE28463E
:1018B00000F040FD28B3237BDFF894B0002B14BF69
:1018C000032302238BF8053000F078FA4FF47A7383
:1018D0005146B0FBF3F0CBF800005846FFF7EAFAA8
:1018E000182307300293124B0193C0F3CF0040F24C
:1018F0005513CDE903A0009342464B46284600F01D
:101900001BFD237B2BB1FFF743FA237B002B7FF4D6
:10191000F6AE13B0BDE8F08F94340020A53500205A
:10192000000002408C340020A0350020C03400208C
:10193000A4350020401DA12026812A0BF1C6A7C195
:10194000D068080FD8350020903400208D34002056
:101950007C24002070B50F4B1B780133DBB2012BC8
:101960000C4611D80C4D29684FF47A730E6AA2FB0D
:101970000332014622462846B047844204D1074B31
:1019800000221A70012070BD4FF4FA7002F0A0F925
:101990000020F8E724230020C0370020D4350020A1
:1019A00007B50023024601210DF107008DF807302D
:1019B000FFF7D0FF20B19DF8070003B05DF804FBEE
:1019C0004FF0FF30F9E700000A4608B50421FFF7A1
:1019D000C1FF80F00100C0B2404208BD30B4054CE8
:1019E0002368DD69044B0A46AC460146204630BCFC
:1019F000604700BFC0370020A086010070B502F02C
:101A000017FC094E094D3080002428683388834232
:101A100008D902F007FC2B6804440133B4F5803F79
:101A20002B60F2D370BD00BFD6350020A835002052
:101A300002F0C0BC00F1006000F580300068704723
:101A400000F10060920000F5803002F03FBC000021
:101A5000054B1A68054B1B889B1A834202D9104418
:101A600002F0E0BB00207047A8350020D6350020EA
:101A700038B5074D04462868204402F0DBFB28B93E
:101A800028682044BDE8384002F0ECBB38BD00BFF8
:101A9000A835002010F003030AD1B0F5047F05D269
:101AA00000F10050A0F51040D0F8003818467047FB
:101AB0000023FBE700F10050A0F51040D0F8100A19
:101AC00070470000064991F8243033B10023086ABA
:101AD00081F824300822FFF7B3BF0120704700BF10
:101AE000AC350020014B1868704700BF002004E0AF
:101AF00070B52A4B1B68C3F30B0204461B0C62B182
:101B000040F21340824230D040F2194082422ED03F
:101B100040F2214082422CD10322214D0C2000FBB7
:101B20000252556842F20102934224D0B3F5805F1D
:101B300023D041F20102934221D041F203029342A9
:101B40001FD041F20702934214BF3F233123013CCF
:101B50000C44013D0A46A24215D215F9016F501CF2
:101B60009EB100F8016C0246F5E70122D5E702229A
:101B7000D3E70C4DD6E73323E9E74123E7E75A23C0
:101B8000E5E75923E3E7104605E02C25844215706C
:101B900001D9901C5370401A70BD00BF002004E0B2
:101BA000DC590008B0590008022802BF024B4FF070
:101BB00080429A61704700BF00000240022802BFC5
:101BC000024B4FF480429A61704700BF0000024010
:101BD000022801BF024A536983F48043536170476E
:101BE0000000024010B50023934203D0CC5CC454E3
:101BF0000133F9E710BD000010B5013810F9013FBD
:101C00003BB191F900409C4203D11AB10131013A34
:101C1000F4E71AB191F90020981A10BD1046FCE7BC
:101C200003460246D01A12F9011B0029FAD1704767
:101C300002440346934202D003F8011BFAE77047BF
:101C40002DE9F8431F4D144695F824200746884691
:101C500052BBDFF870909CB395F824302BB920224A
:101C6000FF2148462F62FFF7E3FF95F82400C0F1FB
:101C70000802A24228BF2246D6B24146920005EB96
:101C80008000FFF7AFFF95F82430A41B1E44F6B286
:101C9000082E17449044E4B285F82460DBD1FFF7A6
:101CA00011FF0028D7D108E02B6A03EB820383429F
:101CB000CFD0FFF707FF0028CBD10020BDE8F88385
:101CC0000120FBE7AC350020024B1A78024B1A705A
:101CD000704700BFD43500202423002010B50F4CDE
:101CE0000F4801F00BFB21460D4801F033FB24683F
:101CF0000C48626DD2F8043843F00203C2F804388D
:101D000001F0E6FF0849204601F02AFC626DD2F896
:101D1000043823F00203C2F8043810BDD05A00087A
:101D2000C037002040420F00D85A0008704700001A
:101D30000FB4002004B0704700B59BB0EFF30981E9
:101D400068226846FFF74EFFEFF30583044B9A6B5A
:101D5000DA6A9A6A9A6A9A6A9A6A9A6A9B6AFEE741
:101D600000ED00E000B59BB0EFF309816822684602
:101D7000FFF738FFEFF30583044B9A6B9A6A9A6A70
:101D80009A6A9A6A9A6A9B6AFEE700BF00ED00E0D1
:101D900000B59BB0EFF3098168226846FFF722FF88
:101DA000EFF30583034B5A6B9A6A9A6A9A6A9A6AA6
:101DB0009B6AFEE700ED00E0FEE7000002F034BBA6
:101DC00002F00CBB30B5094D0A4491420DD011F818
:101DD000013B5840082340F30004013B2C4013F022
:101DE000FF0384EA5000F6D1EFE730BD2083B8ED61
:101DF000F7B54FF0FF33DFF854C0DFF854E000EBE5
:101E000081011A4688421CD050F8044B019401AF5E
:101E1000042417F8015B82EA05620825DB181646E0
:101E200005F1FF355241002EBCBF83EA0C0382EA64
:101E30000E0215F0FF05F1D1013C14F0FF04E8D1CA
:101E4000E0E7D843D14303B0F0BD00BF9336EAA921
:101E5000EBE1F0422DE9F041C56915B9C161BDE87A
:101E6000F0814B6823F06047C3F38A464FEAD37E84
:101E7000C3F3807816EA230638BF3E46AC462B46AD
:101E80005A68BEEBD27F22F060440AD0002A18DAEA
:101E9000A40CB44217D19D420FD10D60DEE713466A
:101EA000EEE7A74207D102F08044C2F380724245B8
:101EB0000BD054B1EFE708D2EDE7CCF800100B607F
:101EC000CDE7B44201D0B442E5D81A689C46002A56
:101ED000E5D11960C3E700002DE9F047089D01F046
:101EE00007044FEAD508224405F0070500EBD100AE
:101EF0004FF47F49944201D1BDE8F08704F0070711
:101F000005F0070A57453E4638BF5646C6F1080653
:101F1000111B8E4228BF0E46E10808EBD50E415C2E
:101F200013F80EC0B94029FA06F721FA0AF1FFB2F8
:101F30008CEA010147FA0AF739408CEA010C03F8F0
:101F40000EC034443544D5E780EA0120082341F22D
:101F5000210201B24000002980B203F1FF33B8BF73
:101F6000504013F0FF03F4D17047000038B50C4621
:101F70008D18A54200D138BD14F8011BFFF7E4FF0E
:101F8000F7E7000002684AB113680360C38801895B
:101F900001339BB29942C38038BF0381104670471A
:101FA00070B588B0202204460D4668460021FFF730
:101FB0003FFE20460495FFF7E5FF024658B16B4609
:101FC000054608AE1C4603CCB4422860696023462F
:101FD00005F10805F6D1104608B070BD082817D9DC
:101FE00009280CD00A280CD00B280CD00C280CD0B7
:101FF0000D280CD00E2814BF4020302070470C2034
:102000007047102070471420704718207047202018
:1020100070470000082817D90C280CD910280CD9B3
:1020200014280CD918280CD920280CD930288CBF9A
:102030000F200E207047092070470A2070470B20A0
:1020400070470C2070470D207047000010B54B689A
:1020500023B9CA8A63F30902CA8210BDC4681A6828
:102060001C60C360438A013B43824A60EFE7000083
:102070002DE9F84F1D46CB8A0F46C3F30901062907
:10208000814692460B4630D00020AAB207F11904CF
:102090009EB2052E1FFA80F80FD8904503F1010378
:1020A00006D3FB8A0A4462F30903FB8201201AE08B
:1020B0001AF80060E6540130EAE79045F1D2A1F148
:1020C000060B1C237C68BBFBF3F203FB12BB1FFA5D
:1020D0008BF6002C45D14846FFF754FF044638B92B
:1020E00078606FF00200BDE8F88F4FF00008E6E777
:1020F000002606607860ADB24FF0000B454510D960
:102100000AEB0803221D13F8011B9155B1B208F127
:1021100001081B291FFA88F82BD0454506F1010656
:10212000F1D8FB8AC3F30902154465F30903BCE740
:10213000013292B21C462368002BF9D1AB1F0B442D
:102140001C21B3FBF1F301339BB29A42D3D2BBF112
:10215000000FD0D14846FFF715FF20B9C4F800B0F2
:10216000BFE70122E7E7C0F800B05E462060044602
:10217000C1E74545D5D94846FFF704FF08B92060B7
:10218000AFE7C0F800B0002620600446B6E70000C4
:102190002DE9F04F2DED028B83B0CDE90013BDF892
:1021A0003C5007469146002A00F092802DB10E9BCC
:1021B000002B00F08D80072D32D807F10C00FFF7BF
:1021C000E1FE044638B96FF00204204603B0BDECCE
:1021D000028BBDE8F08F14220021FFF729FD0E9934
:1021E0002A4604F10800FFF7FDFC681CC0B2FFF7A7
:1021F00011FFFFF7F3FE207499F80030013814FA4C
:1022000080F003F01F0363F03F030372009B43F071
:102210000041616038462146FFF71CFE0124D4E7E7
:1022200000F10C034FF0000808EE103A4FF0800A5E
:102230004646444618EE100AFFF7A4FE83460028DF
:10224000C1D014220021FFF7F3FCC6BB019BABF801
:10225000083002200E9B00F1080299195BFA82F205
:102260000130C0B2082801D0AE422AD3FFF7D2FE17
:10227000FFF7B4FE99F80020009B411E02F01F02F8
:1022800042EA4812AE4208BF4FF0400A5BFA81F1C1
:102290004AEA020A43F0004281F808A08BF81000D5
:1022A000CBF8042059463846FFF7D4FD0134AE423E
:1022B00024B288F001084FF0000ABBD185E7002066
:1022C000C8E711F801CB02F801CB0136B6B2C7E777
:1022D0006FF0010479E70000F8B515460E46282294
:1022E000002104461F46FFF7A3FC069B6360B5F57B
:1022F000001F079BA76034BF6A094FF6FF72236275
:1023000004F10C0097B200239A4205D80023036021
:1023100027826382A382F8BD0660013330462036EF
:10232000F2E7000003781BB94BB2002BC8BF017065
:1023300070470000007870472DE9F74FDDF83C90BA
:10234000BDF830500D9E9DF83840BDF84070804675
:1023500092469B46B9F1000F01D1002F51D11F2C9D
:102360004FD898F80000B0B9072F47D835F00303CD
:1023700047D13A4649464FF6FF70FFF7F7FD20F088
:1023800001002D02400445EA0464400C44EA402464
:102390004FF6FF7321E040EA0520072F40EA04646E
:1023A000F6D900254FF6FF73C5F12000A5F12002F4
:1023B0002AFA05F10BFA00F001432BFA02F211435D
:1023C0001846C9B2FFF7C0FD0835402D0346EBD1D2
:1023D0003A464946FFF7CAFD0346CDE90097324623
:1023E00021464046FFF7D4FE33780133DBB21F2B82
:1023F00088BF0023337003B0BDE8F08F6FF0030097
:10240000F9E76FF00100F6E72DE9F04F85B092464D
:10241000DDF848800F9D9DF840209DF84490BDF860
:102420004C7006469B46B8F1000F01D1002F48D1F1
:102430001F2A46D83378002B46D00C0244EA0264A7
:102440009DF8381044EAC93444EA01441C43072F7C
:1024500044F0800432D900234FF6FF72C3F1200C00
:10246000A3F120002AFA03F10BFA0CFC41EA0C015B
:102470002BFA00F00143C9B210460393FFF764FD45
:10248000039B0833402B0246E8D13A464146FFF70A
:102490006DFD0346CDE900872A4621463046FFF709
:1024A00077FEB9F1010F06D12B780133DBB21F2B78
:1024B00088BF00232B7005B0BDE8F08F4FF6FF7387
:1024C000E8E76FF00100F6E76FF00300F3E70000C4
:1024D000C06900B104307047C3691A68C261C2683C
:1024E0001A60C360438A013B438270472DE9F04183
:1024F000D0F81880194E14461D464146002709B9E8
:10250000BDE8F081D1E90223A21A65EB03039642EC
:1025100077EB03031ED283698B420DD1FFF796FD43
:1025200083691B688361C3680B60438AC1608169EA
:10253000013B43828846E2E7FFF788FD0B68C8F855
:102540000030C3680B60438AC160013B4382D8F806
:102550000010D4E788460968D1E700BF80841E00D8
:102560002DE9F04F8BB00D46DDF8509014469B4698
:102570008046002800F01981B9F1000F00F01581A4
:10258000531E3F2B00F21181012A03D1BBF1000F32
:1025900040F00B810023CDE90833B8F81430B5EBD7
:1025A000C30F4FEAC30703D300200BB0BDE8F08F81
:1025B0002B199F42D8F80C303ABF7F1BFFB2274639
:1025C0001BB9D8F81030002B7AD02F2D4ED8C5F17A
:1025D0003006B7424FF000032CBFF6B23E460093E0
:1025E0002946D8F8080008AB3246FFF775FCA7EB80
:1025F000060A35445FFA8AFAB8F8143003F100533A
:10260000063BDB000493D8F80C3003933021039B86
:1026100013B1BAF1000F2CD1D8F8100040B1BAF1C3
:10262000000F05D0009608AB5246691AFFF754FC1C
:1026300038B2002FB8D066070AD00AAB03EBD4013A
:10264000624211F8083C02F00702134101F8083C0D
:10265000082C3CD9102C40F2B580202C40F2B780D9
:10266000BBF1000F00F09C80082334E0BA4600263E
:10267000C2E7049BE02B28BFE02306930B44AB4248
:10268000059314D95A1B03980096924534BF5246BD
:10269000D2B2691A08AB04300792FFF71DFC079A03
:1026A0001644AAEB020A1544F6B25FFA8AFA049BB2
:1026B000069A05999B1A0493039B1B680393A6E74C
:1026C0000093D8F8080008AB3A462946AEE7BBF1BC
:1026D000000F13D00123B4EBC30F6CD0082C12D819
:1026E0009DF82030621E23FA02F2D50706D54FF07E
:1026F000FF3202FA04F423438DF820309DF8203095
:1027000089F8003051E7102C12D8BDF82030621E35
:1027100023FA02F2D10706D54FF0FF3202FA04F491
:102720002343ADF82030BDF82030A9F800303CE755
:10273000202C0FD80899631E21FA03F3DA0705D578
:102740004FF0FF3202FA04F40C430894089BC9F8D6
:1027500000302AE7402C2BD0DDE90865611EC4F16A
:102760002102A4F1210326FA01F105FA02F225FA69
:1027700003F311431943CB0712D50122A4F120031F
:10278000C4F1200102FA03F322FA01F1A2405242FD
:1027900043EA010363EB430332432B43CDE90823B0
:1027A000DDE90823C9E90023FFE66FF00100FCE63C
:1027B0006FF00800F9E6082CA0D9102CB3D9202C12
:1027C000EED8C3E7BBF1000FADD0022383E7BBF126
:1027D000000FBBD004237EE730B5012A144638BF72
:1027E0000124402C85B028BF40240025012ACDE9D2
:1027F000025518D81B788DF8083063070AD004AB4F
:1028000003EBD405624215F8083C02F0070293403E
:1028100005F8083C009103462246002102A8FFF774
:102820005BFB05B030BD082AE4D9102A03D81B8809
:10283000ADF80830E1E7202A8DBFD3E900231B68FB
:102840000293CDE90223D8E710B5CB681BB98B60A2
:102850000B618B8210BDC4681A681C60C360438A18
:10286000013B4382CA60F0E72DE9F04FD1F80080C8
:1028700093B018F0800FCDE90323C8F3C01219BF3D
:10288000C8F3C03BC8F306264FF0020B1646B8F15A
:10289000000F04460D4680F2D18118F0C043059325
:1028A00040F0CC810B7B002B00F0C881BBF1020F04
:1028B00003D00178B14240F0C48108F07F01069155
:1028C0006AB3C8F3074A2B44069A93F80390760636
:1028D00046EA0B4646EA82465FEAD91346EA0A060A
:1028E000079300F0908000220023CDE90A23069B85
:1028F000009367685B4652460AA92046B8470028FD
:102900007ED0A7699FB9314604F10C00FFF748FB60
:102910000746E0B96FF0020013B0BDE8F08FC8F3CE
:102920000F2A18F07F0F08BF0AF0030ACBE73B69B4
:102930009E420DD03F68002FF9D1314604F10C00C2
:10294000FFF72EFB07460028E4D0A3693B60A76190
:10295000DDE90A2300264FF6FF70C6F1200E22FAA9
:1029600006F103FA0EFEA6F1200C23FA0CFC41EA54
:102970000E0141EA0C01C9B2083609920893FFF72B
:10298000E3FA402EDDE90832E7D1B882FB7D09F099
:102990001F06C3F384039B1BD7E9022198B2002BC7
:1029A000BCBF00F120031BB252EA0100C8F3046867
:1029B0000FD00398821A049860EB0101A748904257
:1029C0004FF000028A4104D3079A002A5BD0012B02
:1029D00023DDFA7D4FEA890302F0030203F07C0352
:1029E0001343FB7539462046FFF730FB079BA3B91D
:1029F000FB7DC3F38402013262F38603FB7504E0BE
:102A00006FF00B0088E7A76917B96FF00C0083E738
:102A10003B699E42BAD03F68F6E719F0400F32D0CA
:102A2000039BBB60049BFB60142200210DA8FFF7F1
:102A3000FFF8039B0A93049B0B932B1D0C932B7B9A
:102A4000ADF83EA0013BDBB2ADF83C30069B8DF803
:102A5000433094F824308DF840B083F001038DF8B2
:102A600044308DF84160A3688DF842800AA9204661
:102A70009847FB7DC3F38403013303F01F039B02DC
:102A8000FB82002048E7FB7DC9F34012B2EBD31F65
:102A900040F0DA80C3F38403B34240F0D880079952
:102AA0002B7B4FEA9912002934D0D20741D4032B53
:102AB00040F2D080039BBB60049BFB602B7BAE1D70
:102AC000033BDBB23246394604F10C00FFF7D0FA83
:102AD00000280DDA20463946FFF7B8FAFB7DC3F32C
:102AE0008403013303F01F039B02FB82032013E7DF
:102AF000AB883B832A7B033AB88AD2B23146FFF7D0
:102B000035FAFB7DB882DA43C2F3C01262F3C71311
:102B1000FB75B6E76AB92E1D013BDBB2324639467A
:102B200004F10C00FFF7A4FA0028D3DB2A7B013A5A
:102B3000E2E7F98AC1F30901013B0529DAB259D864
:102B4000281D002307F11A0C9A4208D910F801EB4E
:102B50000CF801E0013101330629DBB2F4D103990D
:102B60000A9104990B91934207F11A010C9138BF15
:102B7000043379680D9134BF55FA83F300230E9323
:102B8000FB8AADF83EA0C3F309031A44069B8DF8F7
:102B9000433094F82430ADF83C2083F001038DF8E5
:102BA000443000238DF840B08DF841608DF84280AC
:102BB0007B602A7BB88A013A291DFFF7D7F93B8B46
:102BC000B882834203D1A3680AA9204698472046C9
:102BD0000AA9FFF739FEFB7DB88AC3F384030133EA
:102BE00003F01F039B02FB823B8B984214BF112012
:102BF000002091E67B68002BB1D0062001E01C305C
:102C00006346D3F800C0BCF1000FF8D1091A081DC3
:102C100005F1040C00EB030905989DF8143001EB55
:102C2000000EBEF11B0F9AD89A4298D91CF8013BAE
:102C300009F8013B059B01330593EDE76FF00900AF
:102C40006AE66FF00A0067E66FF00D0064E66FF069
:102C50000E0061E66FF00F005EE600BF80841E008C
:102C6000404BF0B51C6C404E44F000741C641D6E6B
:102C700045F000751D661B6E3C4B9B6AD3F80052F5
:102C8000354045F00105C3F80052D3F80042344006
:102C900044EA002040F00100C3F80002002952D0AD
:102CA0000020C3F81C020546C3F80402C3F80C0256
:102CB000C3F8140203EBC00401301C28C4F84052CE
:102CC000C4F84452F6D100254FF0010C96781488D0
:102CD000F70748BFD3F804720CFA04F044BF074367
:102CE000C3F80472B70742BFD3F80C720743C3F8A6
:102CF0000C72760742BFD3F814620643C3F814621D
:102D000003EBC4045668C4F840629668C4F8446291
:102D1000D3F81C4201352043A942C3F81C0202F13A
:102D20000C02D3D1D3F8002222F00102C3F8002212
:102D30000C4B1A6C22F000721A641A6E22F00072A8
:102D40001A661B6EF0BD0122C3F84012C3F844128C
:102D5000C3F80412C3F81412C3F80C22C3F81C22DF
:102D6000E0E700BF003802400000FFFFD835002038
:102D7000184A916A08B58B688B6013F0010104D082
:102D800013F00C0F18BF4FF48031D80506D513F49B
:102D9000406F14BF41F4003141F00201D80306D561
:102DA00013F4402F14BF41F4802141F00401D36992
:102DB0000BB108489847202383F311880648002167
:102DC00000F0AEFF002383F31188BDE8084001F056
:102DD00023BC00BFD8350020E035002038B5124CA8
:102DE000A36ADD68AA0712D05A6922F002025A616A
:102DF000A36913B1012120469847202383F311884A
:102E00000A48002100F08CFF002383F31188EB06B1
:102E100006D5A36A1021D960236A0BB102489847EE
:102E2000BDE8384001F0F8BBD8350020E835002077
:102E300038B5124CA36A1D69AA0712D05A6922F04C
:102E400010025A61A36913B102212046984720233A
:102E500083F311880A48002100F062FF002383F306
:102E60001188EB0606D5A36A10211961236A0BB1FC
:102E700002489847BDE8384001F0CEBBD835002065
:102E8000E835002038B50F4CA36A5D685D602A07FD
:102E90000AD5042222701A6822F002021A60636ABC
:102EA00013B10021204698476B0706D5A36A99699C
:102EB000236A13B1034809049847BDE8384001F07C
:102EC000ABBB00BFD835002010B50E4C204600F03B
:102ED00029F90D4BA3620B21132000F00BF90B21F4
:102EE000142000F007F90B21152000F003F90B2145
:102EF000162000F0FFF80022BDE8104011460E2019
:102F0000FFF7AEBED835002000640040114B984258
:102F100010B5044609D1104B1A6C42F000721A64C5
:102F20001A6E42F000721A661B6EA36A01221A60C2
:102F3000A36A5A68D20707D5626851681268D961D6
:102F40001A60064A5A6110BD0121082000F0D4FD24
:102F5000EEE700BFD8350020003802405B87010053
:102F600003291AD8DFE801F0020A0F14836A9B686C
:102F700013F0E05F14BF012000207047836A986857
:102F8000C0F380607047836A9868C0F3C060704780
:102F9000836A9868C0F30070704700207047000093
:102FA00010B5032925D8DFE801F00225292D836A11
:102FB0009968C1F30161183103EB0113107884069D
:102FC0004CBF54689488C0F300114FEA410148BFD8
:102FD00041EAC40100F00F004CBF41F0040141EA96
:102FE0004451586041F001019068D2689860DA60FD
:102FF000196010BD836A03F5C073DFE7836A03F5C8
:10300000C873DBE7836A03F5D073D7E701290AD0D9
:1030100002290FD081B9836ADA68920701D1186951
:1030200003E001207047836AD86810F0030018BFDE
:1030300001207047836AF2E70020704710B539B964
:10304000836AD96889071BD11B699C0704D110BD0D
:10305000012915D00229FAD1816AD1F8C031D1F8FD
:10306000C441D1F8C8011061D1F8CC0150612020D1
:1030700008610869800717D1486940F0100012E024
:10308000816AD1F8B031D1F8B441D1F8B8011061FA
:10309000D1F8BC0150612020C860C868800703D106
:1030A000486940F002004861C3F34000C3F3800167
:1030B000000140EA4111107920F030000143117104
:1030C00089064BBF91681189DB085B0D4CBF63F328
:1030D0001C0163F30A01137948BF916064F3030391
:1030E00013714FEA14234FEA144458BF118113702F
:1030F0005480ACE700F1604303F561430901C9B2B4
:1031000083F80013012200F01F039A4043099B003B
:1031100003F1604303F56143C3F880211A607047EF
:10312000FFF7D2BE012300F10802C0E902220370BA
:1031300000F110020023C0E90422C0E90633C0E90F
:10314000083343607047000010B52023044683F322
:103150001188022303704160FFF7D8FE0423237017
:10316000002383F3118810BD2DE9F0411F4604466A
:103170000D461646202383F3118800F108082378B2
:10318000052B0DD029462046FFF7EAFE40B1204628
:1031900032462946FFF704FF002080F3118808E03B
:1031A0003946404600F0A0FD0028E8D0002383F314
:1031B0001188BDE8F08100002DE9F0411F4604466A
:1031C0000D461646202383F3118800F1100823785A
:1031D000052B0DD029462046FFF718FF40B12046A9
:1031E00032462946FFF72AFF002080F3118808E0C5
:1031F0003946404600F078FD0028E8D0002383F3EC
:103200001188BDE8F0810000026843681143016045
:1032100003B118477047000013B5446BD4F89434D9
:103220001A681178042915D1217C022912D1197943
:10323000128901238B4013420CD101A904F14C00E7
:1032400001F0A8FFD4F89444019B2179024620683C
:1032500000F0CEF902B010BD143001F02BBF000019
:103260004FF0FF33143001F025BF00004C3001F067
:10327000FDBF00004FF0FF334C3001F0F7BF0000FE
:10328000143001F0F9BE00004FF0FF31143001F0AE
:10329000F3BE00004C3001F0C9BF00004FF0FF3218
:1032A0004C3001F0C3BF00000020704710B5D0F8CB
:1032B00094341A6811780429044617D1017C022934
:1032C00014D15979528901238B4013420ED1143005
:1032D00001F08CFE024648B1D4F894444FF4807358
:1032E00061792068BDE8104000F070B910BD0000A1
:1032F000406BFFF7DBBF0000704700007FB5124B4B
:10330000036000234360C0E90233012502260F4B0E
:10331000057404460290019300F184022946009648
:103320004FF48073143001F03DFE094B0294CDE957
:10333000006304F523724FF48073294604F14C00B6
:1033400001F004FF04B070BD0C5A0008F13200080F
:10335000193200080B68202282F311880A7903EBE6
:10336000820290614A79093243F822008A7912B1C7
:1033700003EB8203986102230374C0F894140023C2
:1033800083F311887047000038B5037F044613B1FA
:1033900090F85430ABB9201D01250221FFF734FF0E
:1033A00004F1140025776FF0010100F0B9FC84F8F6
:1033B000545004F14C006FF00101BDE8384000F0BA
:1033C000AFBC38BD10B5012104460430FFF71CFF27
:1033D0000023237784F8543010BD000038B504462C
:1033E0000025143001F0F6FD04F14C00257701F0C2
:1033F000C5FE201D84F854500121FFF705FF20462B
:10340000BDE83840FFF752BF90F8443003F0600346
:10341000202B07D190F84520212A4FF0000303D834
:103420001F2A06D800207047222AFBD1C0E90E339C
:1034300003E0034A82630722C263036401207047EA
:103440002523002037B5D0F894341A681178042960
:1034500004461AD1017C022917D119791289012356
:103460008B40134211D100F14C05284601F046FF74
:1034700058B101A9284601F08DFED4F89444019B6F
:1034800021790246206800F0B3F803B030BD000097
:10349000F0B500EB810385B09E6904460D46FEB190
:1034A000202383F3118804EB8507301D0821FFF7E3
:1034B000ABFEFB685B691B6806F14C001BB1019019
:1034C00001F076FE019803A901F064FE024648B1BE
:1034D000039B2946204600F08BF8002383F31188D4
:1034E00005B0F0BDFB685A691268002AF5D01B8A46
:1034F000013B1340F1D104F14402EAE7093138B548
:1035000050F82140DCB1202383F31188D4F89424AF
:103510001368527903EB8203DB689B695D6845B1F0
:1035200004216018FFF770FE294604F1140001F031
:1035300067FD2046FFF7BAFE002383F3118838BDEC
:103540007047000001F02AB9012303700023C0E98D
:103550000133C36183620362C362436203637047E2
:1035600038B50446202383F311880025C0E90355AC
:10357000C0E90555416001F021F90223237085F36C
:10358000118838BD70B500EB810305465069DA60DB
:103590000E46144618B110220021FEF749FBA0691F
:1035A00018B110220021FEF743FB31462846BDE842
:1035B000704001F0CDB90000826802F00112826013
:1035C0000022C0E90422826101F04EBAF0B400EB9F
:1035D00081044789E4680125A4698D403D43458104
:1035E00023600023A2606360F0BC01F069BA0000B0
:1035F000F0B400EB81040789E468012564698D401B
:103600003D43058123600023A2606360F0BC01F0AC
:10361000E3BA000070B50223002504460370C0E938
:103620000255C0E90455C564856180F8345001F045
:103630002BF963681B6823B129462046BDE870401A
:10364000184770BD037880F8503005230370436835
:103650001B6810B504460BB1042198470023A360F2
:1036600010BD000090F85020436802701B680BB139
:10367000052118477047000070B590F834300446B3
:1036800013B1002380F8343004F14402204601F0E5
:103690000DFA63689B68B3B994F8443013F0600581
:1036A00035D00021204601F05FFC0021204601F0CA
:1036B00051FC63681B6813B1062120469847062316
:1036C00084F8343070BD204698470028E4D0B4F820
:1036D0004A30E26B9A4288BFE36394F94430E56B69
:1036E000002B4FF0200380F20381002D00F0F280C8
:1036F000092284F8342083F311880021D4E90E23B1
:103700002046FFF775FF002383F31188DAE794F86A
:10371000452003F07F0343EA022340F20232934242
:1037200000F0C58021D8B3F5807F48D00DD8012B9B
:103730003FD0022B00F09380002BB2D104F14C0259
:10374000A2630222E2632364C1E7B3F5817F00F044
:103750009B80B3F5407FA4D194F84630012BA0D1D3
:10376000B4F84C3043F0020332E0B3F5006F4DD0B3
:1037700017D8B3F5A06F31D0A3F5C063012B90D853
:10378000636894F846205E6894F84710B4F84830AF
:103790002046B047002884D04368A3630368E363EE
:1037A0001AE0B3F5106F36D040F6024293427FF430
:1037B00078AF5C4BA3630223E3630023C3E794F871
:1037C0004630012B7FF46DAFB4F84C3023F0020388
:1037D000C4E90E55A4F84C30256478E7B4F84430B9
:1037E000B3F5A06F0ED194F8463084F84E302046E1
:1037F00001F0A2F863681B6813B1012120469847C5
:10380000032323700023C4E90E339CE704F14F0324
:10381000A3630123C3E72378042B10D1202383F370
:1038200011882046FFF7C8FE85F3118803216368DD
:1038300084F84F5021701B680BB12046984794F8CC
:103840004630002BDED084F84F30042323706368A9
:103850001B68002BD6D0022120469847D2E794F867
:1038600048301D0603F00F0120460AD501F010F97B
:10387000012804D002287FF414AF2B4B9AE72B4B7E
:1038800098E701F0F7F8F3E794F84630002B7FF45F
:1038900008AF94F8483013F00F01B3D01A06204651
:1038A00002D501F075FBADE701F068FBAAE794F8DB
:1038B0004630002B7FF4F5AE94F8483013F00F013A
:1038C000A0D01B06204602D501F04EFB9AE701F07E
:1038D00041FB97E7142284F8342083F311882B46A8
:1038E0002A4629462046FFF771FE85F31188E9E64E
:1038F0005DB1152284F8342083F311880021D4E9C6
:103900000E232046FFF762FEFDE60B2284F83420EA
:1039100083F311882B462A4629462046FFF768FE86
:10392000E3E700BF3C5A0008345A0008385A000840
:1039300038B590F834300446002B3ED0063BDAB25E
:103940000F2A34D80F2B32D8DFE803F03731310893
:10395000223231313131313131313737C56BB0F845
:103960004A309D4214D2C3681B8AB5FBF3F203FBB5
:1039700012556DB9202383F311882B462A46294618
:10398000FFF736FE85F311880A2384F834300EE001
:10399000142384F83430202383F3118800231A463B
:1039A00019462046FFF712FE002383F3118838BD25
:1039B000036C03B198470023E7E70021204601F09C
:1039C000D3FA0021204601F0C5FA63681B6813B1E1
:1039D0000621204698470623D7E7000010B590F847
:1039E0003430142B044629D017D8062B05D001D823
:1039F0001BB110BD093B022BFBD80021204601F072
:103A0000B3FA0021204601F0A5FA63681B6813B1E0
:103A1000062120469847062319E0152BE9D10B23F0
:103A200080F83430202383F3118800231A46194686
:103A3000FFF7DEFD002383F31188DAE7C3689B6993
:103A40005B68002BD5D1036C03B19847002384F841
:103A50003430CEE7024B0022C3E900339A6070474E
:103A600004360020002303748268054B1B689968A4
:103A70009142FBD25A680360426010605860704700
:103A80000436002008B5202383F31188037C032B20
:103A900005D0042B0DD02BB983F3118808BD4369E1
:103AA00000221A604FF0FF334361FFF7DBFF002372
:103AB000F2E7D0E9003213605A60F3E700230374A1
:103AC0008268054B1B6899689142FBD85A6803606D
:103AD000426010605860704704360020054B196939
:103AE0000874186802681A6053601861012303742F
:103AF000FCF78EBD0436002030B54B1C0B4D87B053
:103B0000044610D02B690A4A01A800F025F9204686
:103B1000FFF7E4FF049B13B101A800F059F92B69EA
:103B2000586907B030BDFFF7D9FFF8E70436002029
:103B3000853A000838B50C4D41612B6981689A6857
:103B40009142044603D8BDE83840FFF78BBF1846C2
:103B5000FFF7B4FF01232C61014623742046BDE822
:103B60003840FCF755BD00BF04360020044B1A68EE
:103B70001B6990689B68984294BF002001207047A1
:103B80000436002010B5084C236820691A682260AA
:103B90005460012223611A74FFF790FF01462069E7
:103BA000BDE81040FCF734BD0436002008B5FFF72F
:103BB000DDFF18B1BDE80840FFF7E4BF08BD000015
:103BC000FFF7E0BFFEE7000010B50C4CFFF742FF27
:103BD00000F0B4F80A498022204600F03BF80123A7
:103BE00044F8180C037400F0F3FC002383F31188ED
:103BF00062B60448BDE8104000F04CB82C360020F6
:103C0000405A0008505A000800F01CB9EFF3118028
:103C100020B9EFF30583202282F31188704700005A
:103C200010B530B9EFF30584C4F3080414B180F380
:103C3000118810BDFFF7BAFF84F31188F9E700007F
:103C4000034A516853685B1A9842FBD8704700BF1B
:103C5000001000E082600222028270478368A3F1B4
:103C60007C0243F80C2C026943F83C2C426943F86F
:103C7000382C074A43F81C2CC26843F8102C022247
:103C800003F8082C002203F8072CA3F11800704752
:103C90002906000810B5202383F31188FFF7DEFF03
:103CA00000210446FFF746FF002383F311882046D6
:103CB00010BD0000024B1B6958610F20FFF70EBFBB
:103CC00004360020202383F31188FFF7F3BF0000A0
:103CD00008B50146202383F311880820FFF70CFF65
:103CE000002383F3118808BD49B1064B42681B6964
:103CF00018605A60136043600420FFF7FDBE4FF068
:103D0000FF307047043600200368984206D01A68D6
:103D10000260506059611846FFF7A4BE704700006A
:103D200038B504460D462068844200D138BD03688A
:103D300023605C604561FFF795FEF4E7054B03F1F6
:103D40001402C3E905224FF0FF310022C3E9071234
:103D5000704700BF0436002070B51C4EC0E9032335
:103D600005460C4601F0FCFA334653F8142F9A42EC
:103D70000DD13062C5E901242A600A2C2CBF00193C
:103D80000A30C6E90555BDE8704001F0D7BA316A7E
:103D9000431AE31838BF1C469368A34202D9081996
:103DA00001F0DAFA73699A6894420CD85A68AC60E8
:103DB0002B606A6015609A685D60121B9A604FF014
:103DC000FF33F36170BD1B68A41AECE704360020D2
:103DD00038B51B4C636998420DD0D0E900321360AE
:103DE0005A6000228168C2609A680A449A604FF063
:103DF000FF33E36138BD2246036842F8143F0021D7
:103E000093425A60C16003D1BDE8384001F09EBAC8
:103E10009A688168256A0A449A6001F0A1FA636988
:103E20009A68411B8A42E5D9AB181D1A092D206AF0
:103E300098BF01F10A02BDE83840104401F08CBA85
:103E4000043600202DE9F041184C002704F1140637
:103E5000656901F085FA236AAA68C11A8A4215D8F1
:103E600013442362D5E9003213605A606369D5F8C0
:103E70000C80EF60B34201D101F068FA87F311883A
:103E80002869C047202383F31188E1E76169B142C3
:103E900009D013441B1ABDE8F0410A2B2CBFC018EF
:103EA0000A3001F059BABDE8F08100BF04360020A5
:103EB00000207047FEE70000704700004FF0FF3021
:103EC0007047000002290CD0032904D001290748BB
:103ED00018BF00207047032A05D8054800EBC20030
:103EE0007047044870470020704700BF345B0008EB
:103EF00034230020E85A000870B59AB005460846F9
:103F000001A9144600F0C2F801A8FDF789FE431C80
:103F10005B00C5E900340022237003236370C6B23E
:103F200001AB02341046D1B28E4204F1020401D832
:103F30001AB070BD13F8011B04F8021C04F8010C40
:103F40000132F0E708B5202383F311880348FFF717
:103F500079FA002383F3118808BD00BFC037002021
:103F600090F8443003F01F02012A07D190F8452051
:103F70000B2A03D10023C0E90E3315E003F06003E0
:103F8000202B08D1B0F848302BB990F84520212AD1
:103F900003D81F2A04D8FFF737BA222AEBD0FAE752
:103FA000034A82630722C26303640120704700BF93
:103FB0002C23002007B5052917D8DFE801F01916D2
:103FC00003191920202383F31188104A019001213D
:103FD000FFF7D8FA01980E4A0221FFF7D3FA0D48ED
:103FE000FFF7FCF9002383F3118803B05DF804FBAD
:103FF000202383F311880748FFF7C6F9F2E720234F
:1040000083F311880348FFF7DDF9EBE7885A0008CE
:10401000AC5A0008C037002038B50C4D0C4C0D4987
:104020002A4604F10800FFF767FF05F1CA0204F110
:1040300010000949FFF760FF05F5CA7204F1180086
:104040000649BDE83840FFF757BF00BF883C002055
:1040500034230020685A0008725A00087D5A00086C
:1040600070B5044608460D46FDF7DAFDC6B2204697
:10407000013403780BB9184670BD32462946FDF766
:10408000BBFD0028F3D10120F6E700002DE9F04741
:1040900005460C46FDF7C4FD2B49C6B22846FFF77E
:1040A000DFFF08B10636F6B228492846FFF7D8FFE9
:1040B00008B11036F6B2632E0BD8DFF88C80DFF82B
:1040C0008C90234FDFF894A02E7846B92670BDE877
:1040D000F08729462046BDE8F04701F005BC252EB3
:1040E0002ED1072241462846FDF786FD70B9194BAF
:1040F000224603F10C0153F8040B42F8040B8B42E7
:10410000F9D11B78137007350D34DDE708224946D5
:104110002846FDF771FD98B90F4BA21C19780909C3
:104120000232C95D02F8041C13F8011B01F00F01F3
:104130005345C95D02F8031CF0D118340835C3E7B4
:1041400004F8016B0135BFE7545B00087D5A000895
:104150006A5B00085C5B0008107AFF1F1C7AFF1F77
:10416000BFF34F8F024AD368DB03FCD4704700BF14
:10417000003C024008B5094B1B7873B9FFF7F0FF0C
:10418000074B1A69002ABFBF064A5A6002F18832FB
:104190005A601A6822F480621A6008BDE63E002068
:1041A000003C02402301674508B50B4B1B7893B9CF
:1041B000FFF7D6FF094B1A6942F000421A611A68EC
:1041C00042F480521A601A6822F480521A601A6807
:1041D00042F480621A6008BDE63E0020003C0240C6
:1041E0000B28F0B516D80C4C0C4923787BB90C4D34
:1041F0000E460C234FF0006255F8047B46F8042B62
:10420000013B13F0FF033A44F6D10123237051F828
:104210002000F0BD0020FCE7183F0020E83E002011
:104220007C5B0008014B53F8200070477C5B000862
:104230000C2070470B2810B5044601D9002010BD92
:10424000FFF7CEFF064B53F824301844C21A0BB9BF
:104250000120F4E712680132F0D1043BF6E700BF19
:104260007C5B00080B2838B5044628D8FFF7CEFC45
:10427000FFF776FFFFF77EFF124AF323D360E300D8
:10428000DBB243F4007343F002031361136943F498
:104290008033136105462046FFF762FFFFF7A0FF5A
:1042A000094B53F8241000F039F92846FFF77CFF3A
:1042B000FFF7B6FC2046BDE83840FFF7BBBF002043
:1042C00038BD00BF003C02407C5B000812F00103D7
:1042D0002DE9F04105460E4614464BD18218B2F145
:1042E000016F61D8314B1B6813F001035CD0304F74
:1042F000FFF78CFCFFF73EFFF323FB60FFF730FF77
:10430000314640F20128032C18D824F00104284E2D
:104310000C446D1A40F20118A142336905EB010704
:104320002AD123F001033361FFF73EFFFFF778FC4A
:104330000120BDE8F081043C0435E4E7AB07E4D19B
:104340003B6923F440733B613B6943EA08033B61EB
:1043500051F8046B2E60BFF34F8FFFF701FF2B68FE
:104360009E42E8D03B6923F001033B61FFF71CFF4D
:10437000FFF756FC0020DCE723F440733361336918
:1043800043EA080333610B883B80BFF34F8FFFF78D
:10439000E7FE3F8831F8023BBFB2BB42BCD0336975
:1043A00023F001033361E1E71846C2E70038024019
:1043B000003C0240084908B50B7828B11BB9FFF74B
:1043C000D9FE01230B7008BD002BFCD0BDE80840CE
:1043D0000870FFF7E9BE00BFE63E002070B582B06E
:1043E000FFF714FC0E4E054600F0BAFF326890420B
:1043F00037BF0C4A0B49516814682EBFD1E9004100
:10440000013151600419034641F100012846019130
:104410003360FFF705FC0199204602B070BD00BF74
:104420001C3F0020203F002070B582B0FFF7EEFB5C
:10443000104E054600F094FF3268904237BF0E4A96
:104440000D49516814682EBFD1E900410131516016
:10445000041941F100010346284601913360FFF73A
:10446000DFFB01994FF47A7200232046FBF7B8FE78
:1044700002B070BD1C3F0020203F002010B5024458
:10448000064BD2B2904200D110BD441C00B253F88A
:10449000200041F8040BE0B2F4E700BF50280040D0
:1044A0000F4B30B51C6F240407D41C6F44F4007408
:1044B0001C671C6F44F400441C670A4C236843F4D7
:1044C000807323600244084BD2B2904200D130BDC9
:1044D000441C00B251F8045B43F82050E0B2F4E70A
:1044E00000380240007000405028004007B501220B
:1044F00001A90020FFF7C2FF019803B05DF804FB9B
:1045000013B50446FFF7F2FFA04205D0012201A92E
:1045100000200194FFF7C4FF02B010BD70470000F7
:10452000074B45F255521A6002225A6040F6FF725C
:104530009A604CF6CC421A60024B01221A70704706
:10454000003000402C3F0020034B1B781BB1034B75
:104550004AF6AA221A6070472C3F00200030004023
:10456000034B1A681AB9034AD2F874281A607047C4
:10457000283F002000300240024B4FF08072C3F809
:10458000742870470030024008B5FFF7E9FF024B7E
:104590001868C0F3407008BD283F002008B5FFF739
:1045A000DFFF024B1868C0F3007008BD283F0020F1
:1045B000EFF3098305494A6B22F001024A6368332D
:1045C00083F30988002383F31188704700EF00E02C
:1045D000202080F3118862B60C4B0D4AD96821F473
:1045E000E0610904090C0A43DA60D3F8FC200949A8
:1045F00042F08072C3F8FC200A6842F001020A60AF
:104600001022DA7783F82200704700BF00ED00E047
:104610000003FA05001000E010B5202383F3118891
:104620000E4B5B6813F4006314D0F1EE103AEFF315
:104630000984683C4FF08073E361094BDB6B2366B0
:1046400084F30988FFF792FA10B1064BA36110BDFD
:10465000054BFBE783F31188F9E700BF00ED00E0AD
:1046600000EF00E03B0600083E060008704700002F
:10467000FEE700000A4B0B480B4A90420BD30B4B52
:10468000DA1C121AC11E22F003028B4238BF00222C
:104690000021FDF7CDBA53F8041B40F8041BECE7EA
:1046A000345D0008284000202840002028400020D9
:1046B0007047000070B5D0E915439E6800224FF0A6
:1046C000FF3504EB42135101D3F800090028BEBFA7
:1046D000D3F8000940F08040C3F80009D3F8000B7C
:1046E0000028BEBFD3F8000B40F08040C3F8000B99
:1046F000013263189642C3F80859C3F8085BE0D248
:104700004FF00113C4F81C3870BD00001D4B03EBC3
:1047100080022DE9F043D2F80CC05D6DDCF8142066
:10472000461CD2F800E005EB063605EB4018516850
:1047300071450AD3D5F83438012202FA00F023EA91
:104740000000C5F83408BDE8F083BCF81040AEEBBB
:104750000103A34228BF2346D8F81849A4B2B3EBFB
:10476000840FF0D89468A4F1040959F8047F3760E5
:10477000A4EB09071F44042FF7D81C440B44946092
:104780005360D4E7303F0020890141F020010161EE
:1047900003699B06FCD41220FFF752BA10B5054CF2
:1047A0002046FEF7D1FE4FF0A0436365024BA365A0
:1047B00010BD00BF303F0020D05B000870B503780B
:1047C000012B054650D12A4B446D98421BD1294BF1
:1047D0005A6B42F080025A635A6D42F080025A6569
:1047E0005A6D5A6942F080025A615A6922F0800279
:1047F0005A610E2143205B69FEF77CFC1E4BE3608F
:104800001E4BC4F800380023C4F8003EC0232360C8
:104810006E6D4FF40413A3633369002BFCDA01239C
:1048200033610C20FFF70CFA3369DB07FCD412204C
:10483000FFF706FA3369002BFCDA0026A66028464B
:10484000FFF738FF6B68C4F81068DB68C4F81468B9
:10485000C4F81C684BB90A4BA3614FF0FF33636186
:10486000A36843F00103A36070BD064BF4E700BFEB
:10487000303F002000380240401400400300200276
:10488000003C30C0083C30C0F8B5446D05460021FE
:104890002046FFF779FFA96D00234FF001128F68C2
:1048A000C4F834384FF00066C4F81C284FF0FF30CD
:1048B00004EB431201339F42C2F80069C2F8006B57
:1048C000C2F80809C2F8080BF2D20B686A6DEB65F2
:1048D000636210231361166916F01006FBD11220D3
:1048E000FFF7AEF9D4F8003823F4FE63C4F80038BB
:1048F000A36943F4402343F01003A3610923C4F8E0
:104900001038C4F814380A4BEB604FF0C043C4F8B9
:10491000103B084BC4F8003BC4F81069C4F80039D8
:10492000EB6D03F1100243F48013EA65A362F8BD56
:10493000AC5B000840800010426D90F84E10D2F839
:10494000003823F4FE6343EA0113C2F800387047CD
:104950002DE9F84300EB8103456DDA68166806F02F
:104960000306731E022B05EB41130C4680460FFA1B
:1049700081F94FEA41104FF00001C3F8101B4FF0CE
:10498000010104F1100398BFB60401FA03F3916921
:104990008EBF334E06F1805606F5004600293AD008
:1049A000578A04F15801490137436F50D5F81C1854
:1049B0000B43C5F81C382B180021C3F81019536994
:1049C0000127611EA7409BB3138A928B9B08012A83
:1049D00088BF5343D8F85C20981842EA034301F19A
:1049E000400205EB8202C8F85C002146536028466D
:1049F000FFF7CAFE08EB8900C3681B8A43EA8453A9
:104A0000483464011E432E51D5F81C381F43C5F8A5
:104A10001C78BDE8F88305EB4917D7F8001B21F493
:104A20000041C7F8001BD5F81C1821EA0303C0E7B2
:104A300004F13F0305EB83030A4A5A6028462146E6
:104A4000FFF7A2FE05EB4910D0F8003923F400432C
:104A5000C0F80039D5F81C3823EA0707D7E700BFAC
:104A60000080001000040002826D1268C265FFF72A
:104A700021BE00005831436D49015B5813F40040DA
:104A800004D013F4001F0CBF022001207047000067
:104A90004831436D49015B5813F4004004D013F4CE
:104AA000001F0CBF022001207047000000EB8101B5
:104AB000CB68196A0B6813604B685360704700003D
:104AC00000EB810330B5DD68AA691368D36019B9BA
:104AD000402B84BF402313606B8A1468426D1C44D2
:104AE000013CB4FBF3F46343033323F0030302EB11
:104AF000411043EAC44343F0C043C0F8103B2B6865
:104B000003F00303012B09B20ED1D2F8083802EBEF
:104B1000411013F4807FD0F8003B14BF43F0805362
:104B200043F00053C0F8003B02EB4112D2F8003BC7
:104B300043F00443C2F8003B30BD00002DE9F041D2
:104B4000244D6E6D06EB40130446D3F8087BC3F882
:104B5000087B38070AD5D6F81438190706D505EBAF
:104B600084032146DB6828465B689847FA071FD50F
:104B7000D6F81438DB071BD505EB8403D968CCB90C
:104B80008B69488A5A68B2FBF0F600FB16228AB994
:104B90001868DA6890420DD2121AC3E90024202363
:104BA00083F311880B482146FFF78AFF84F31188AD
:104BB000BDE8F081012303FA04F26B8923EA0203C2
:104BC0006B81CB68002BF3D021460248BDE8F04151
:104BD000184700BF303F002000EB810370B5DD684F
:104BE000436D6C692668E6604A0156BB1A444FF46F
:104BF0000020C2F810092A6802F00302012A0AB252
:104C00000ED1D3F8080803EB421410F4807FD4F8D7
:104C1000000914BF40F0805040F00050C4F8000973
:104C200003EB4212D2F8000940F00440C2F8000938
:104C3000D3F83408012202FA01F10143C3F8341811
:104C400070BD19B9402E84BF4020206020682E8A94
:104C50008419013CB4FBF6F440EAC44040F0005033
:104C60001A44C6E7F8B504461E48456D05EB4413E3
:104C7000D3F80869C3F80869F10717D5D5F81038D3
:104C8000DA0713D500EB8403D9684B691F68DA682B
:104C9000974218D2D21B00271A605F60202383F34B
:104CA00011882146FFF798FF87F31188330617D53F
:104CB000D5F834280123A340134211D02046BDE883
:104CC000F840FFF723BD012303FA04F2038923EA26
:104CD000020303818B68002BE8D021469847E5E763
:104CE000F8BD00BF303F00202DE9F74F984C666DAE
:104CF0007569B3691D4015F48058756107D0204669
:104D0000FEF788FC03B0BDE8F04FFFF785BC002D2F
:104D100012DAD6F8003E8E489F071EBFD6F8003E36
:104D200023F00303C6F8003ED6F8043823F001034D
:104D3000C6F80438FEF796FC280505D58448FFF729
:104D4000B9FC8348FEF77EFCA9040CD5D6F80838D8
:104D500013F0060FF36823F470530CBF43F41053A1
:104D600043F4A053F3602A0704D56368DB680BB1F2
:104D700077489847EB0274D4AF0227D5D4F8549003
:104D8000DFF8CCB100274FF0010A09EB4712D2F847
:104D9000003B03F44023B3F5802F11D1D2F8003B40
:104DA000002B0DDA62890AFA07F322EA0303638112
:104DB00004EB8703DB68DB6813B139465846984734
:104DC000A36D01379B68FFB29F42DED9E80617D575
:104DD000676D3A6AC2F30A1002F00F0302F4F01290
:104DE000B2F5802F00F08880B2F5402F08D104EB97
:104DF00083030022DB681B6A07F5805790426DD160
:104E00002903D6F8184813D5E20302D50020FFF78E
:104E100095FEA30302D50120FFF790FE670302D59C
:104E20000220FFF78BFE260302D50320FFF786FE44
:104E30006D037FF567AFE00702D50020FFF712FF93
:104E4000A10702D50120FFF70DFF620702D502205E
:104E5000FFF708FF23077FF555AF0320FFF702FF99
:104E600050E7636DDFF8E8B0019300274FF0010AC7
:104E7000A36D9B685FFA87F999453FF67DAF019B6B
:104E800003EB4913D3F8002902F44022B2F5802F36
:104E900022D1D3F80029002A1EDAD3F8002942F0E3
:104EA0009042C3F80029D3F80029002AFBDB606D8B
:104EB0004946FFF769FC22890AFA09F322EA03034B
:104EC000238104EB8903DB689B6813B1494658468C
:104ED00098474846FFF71AFC0137C9E7910708BF12
:104EE000D7F80080072A98BF03F8018B02F101026E
:104EF00098BF4FEA182881E7023304EB830207F5D5
:104F000080575268D2F818C0DCF80820DCE9001C91
:104F1000A1EB0C0C002188420AD104EB83046368E6
:104F20009B699A6802449A605A6802445A6067E72B
:104F300011F0030F08BFD7F800808C4588BF02F836
:104F4000018B01F1010188BF4FEA1828E3E700BF98
:104F5000303F0020436D03EB4111D1F8003B43F497
:104F60000013C1F8003B7047436D03EB4111D1F8CA
:104F7000003943F40013C1F800397047436D03EB67
:104F80004111D1F8003B23F40013C1F8003B7047F6
:104F9000436D03EB4111D1F8003923F40013C1F83C
:104FA0000039704730B5039C0172043304FB0325BC
:104FB000C0E90653049B03630021059BC160C0E95F
:104FC0000000C0E90422C0E90842C0E90A114363B5
:104FD00030BD0000416A0022C0E90411C0E90A2284
:104FE000C2606FF00101FEF79BBE0000D0E9043201
:104FF000934201D1C2680AB9181D7047002070475A
:1050000003691960C2680132C260C26913448269CF
:105010000361934224BF436A03610021FEF774BE1B
:1050200038B504460D46E3683BB16269131D12684A
:10503000A3621344E362002007E0237A33B92946D0
:105040002046FEF751FE0028EDDA38BD6FF0010072
:10505000FBE70000C368C269013BC36043691344B6
:1050600082694361934224BF436A436100238362A0
:10507000036B03B11847704770B52023044683F3D0
:105080001188866A3EB9FFF7CBFF054618B186F353
:105090001188284670BDA36AE26A13F8015BA36217
:1050A000934202D32046FFF7D5FF002383F31188F4
:1050B000EFE700002DE9F84F04460E4617469846E4
:1050C0004FF0200989F311880025AA46D4F828B0AA
:1050D000BBF1000F09D141462046FFF7A1FF20B1E7
:1050E0008BF311882846BDE8F88FD4E90A12A7EBA4
:1050F000050B521A934528BF9346BBF1400F1BD9AD
:10510000334601F1400251F8040B43F8040B91427D
:10511000F9D1A36A40334036A3624035D4E90A236B
:105120009A4202D32046FFF795FF8AF31188BD42C9
:10513000D8D289F31188C9E730465A46FCF752FDA8
:10514000A36A5B445E44A3625D44E7E710B5029C3A
:105150000172043304FB0321C0E906130023C0E9F4
:105160000A33039B0363049BC460C0E90000C0E9E9
:105170000422C0E90842436310BD0000026AC26015
:10518000426AC0E904220022C0E90A226FF001014C
:10519000FEF7C6BDD0E904239A4201D1C26822B904
:1051A000184650F8043B0B60704700207047000021
:1051B000C368C2690133C3604369134482694361B0
:1051C000934224BF436A43610021FEF79DBD000066
:1051D00038B504460D46E3683BB123691A1DA26247
:1051E000E2691344E362002007E0237A33B92946D9
:1051F0002046FEF779FD0028EDDA38BD6FF001009A
:10520000FBE7000003691960C268013AC260C26925
:10521000134482690361934224BF436A03610023FC
:105220008362036B03B118477047000070B52023F9
:105230000D460446114683F31188866A2EB9FFF79E
:10524000C7FF10B186F3118870BDA36A1D70A36AF1
:10525000E26A01339342A36204D3E1692046043930
:10526000FFF7D0FF002080F31188EDE72DE9F84F1C
:1052700004460D46904699464FF0200A8AF311885D
:105280000026B346A76A4FB949462046FFF7A0FF5C
:1052900020B187F311883046BDE8F88FD4E90A07BA
:1052A0003A1AA8EB0607974228BF1746402F1BD98A
:1052B00005F1400355F8042B40F8042B9D42F9D129
:1052C000A36A4033A3624036D4E90A239A4204D346
:1052D000E16920460439FFF795FF8BF311884645B5
:1052E000D9D28AF31188CDE729463A46FCF77AFCF1
:1052F000A36A3B443D44A3623E44E5E7D0E904236E
:105300009A4217D1C3689BB1836A8BB1043B9B1A45
:105310000ED01360C368013BC360C3691A4483693C
:1053200002619A4224BF436A03610023836201231E
:10533000184670470023FBE700F088B84FF0804321
:10534000002258631A610222DA6070474FF08043EE
:105350000022DA60704700004FF0804358637047C6
:105360004FF08043586A70474B6843608B68836096
:10537000CB68C3600B6943614B6903628B6943620D
:105380000B6803607047000008B5264B26481A6971
:1053900040F2FF110A431A611A6922F4FF7222F0E7
:1053A00001021A611A691A6B0A431A631A6D0A43D9
:1053B0001A651E4A1B6D1146FFF7D6FF02F11C014C
:1053C00000F58060FFF7D0FF02F1380100F5806042
:1053D000FFF7CAFF02F1540100F58060FFF7C4FF38
:1053E00002F1700100F58060FFF7BEFF02F18C0151
:1053F00000F58060FFF7B8FF02F1A80100F58060BA
:10540000FFF7B2FF02F1C40100F58060FFF7ACFFC7
:1054100002F1E00100F58060FFF7A6FFBDE808405B
:1054200000F09AB80038024000000240DC5B00083F
:1054300008B500F007FAFEF7C7FBFFF791F8BDE8E3
:105440000840FEF7E9BD000070470000104B1A6CE1
:1054500042F001021A641A6E42F001021A660D4A05
:105460001B6E936843F0010393604FF08043532217
:105470009A624FF0FF32DA6200229A615A63DA6070
:105480005A6001225A6108211A601C20FDF732BEC1
:1054900000380240002004E04FF0804208B5116956
:1054A000D3680B40D9B2C9439B07116107D52023AC
:1054B00083F31188FEF7A8FB002383F3118808BD4E
:1054C00008B5FFF7E9FFBDE80840FFF7A5B8000001
:1054D0001F4B1A696FEAC2526FEAD2521A611A69F7
:1054E000C2F308021A614FF0FF301A695A69586115
:1054F00000215A6959615A691A6A62F080521A6227
:105500001A6A02F080521A621A6A5A6A58625A6A11
:1055100059625A6A1A6C42F080521A641A6E42F04A
:1055200080521A661A6E0B4A106840F48070106040
:10553000186F00F44070B0F5007F1EBF4FF480304C
:1055400018671967536823F40073536000F05AB961
:105550000038024000700040334B4FF080521A6414
:10556000324A4FF4404111601A6842F001021A6059
:105570001A689107FCD59A6822F003029A602A4BB8
:105580009A6812F00C02FBD1196801F0F901196058
:105590009A601A6842F480321A601A689203FCD545
:1055A0005A6F42F001025A671F4B5A6F9007FCD5A1
:1055B0001F4A5A601A6842F080721A601B4A536888
:1055C0005904FCD5184B1A689201FCD5194A9A6007
:1055D000194B1A68194B9A42194B21D1194A116873
:1055E000194A91421CD140F205121A60144A1368FC
:1055F00003F00F03052BFAD10B4B9A6842F002021D
:105600009A609A6802F00C02082AFAD15A6C42F4A5
:1056100080425A645A6E42F480425A665B6E70470A
:1056200040F20572E1E700BF003802400070004020
:105630000854400700948838002004E011640020DA
:10564000003C024000ED00E041C20F41084A08B5AD
:10565000516913680B4003F00103536123B1054AFC
:1056600013680BB150689847BDE80840FEF7D4BFF7
:10567000003C0140A83F0020084A08B55169136862
:105680000B4003F00203536123B1054A93680BB149
:10569000D0689847BDE80840FEF7BEBF003C014017
:1056A000A83F0020084A08B5516913680B4003F071
:1056B0000403536123B1054A13690BB1506998473C
:1056C000BDE80840FEF7A8BF003C0140A83F00200D
:1056D000084A08B5516913680B4003F00803536189
:1056E00023B1054A93690BB1D0699847BDE80840DA
:1056F000FEF792BF003C0140A83F0020084A08B5D1
:10570000516913680B4003F01003536123B1054A3C
:10571000136A0BB1506A9847BDE80840FEF77CBF9A
:10572000003C0140A83F0020174B10B55A691C6887
:10573000144004F478725A61A30604D5134A936A9C
:105740000BB1D06A9847600604D5104A136B0BB1B1
:10575000506B9847210604D50C4A936B0BB1D06B64
:105760009847E20504D5094A136C0BB1506C984771
:10577000A30504D5054A936C0BB1D06C9847BDE8DE
:105780001040FEF749BF00BF003C0140A83F002089
:105790001A4B10B55A691C68144004F47C425A61D3
:1057A000620504D5164A136D0BB1506D9847230559
:1057B00004D5134A936D0BB1D06D9847E00404D51E
:1057C0000F4A136E0BB1506E9847A10404D50C4AD2
:1057D000936E0BB1D06E9847620404D5084A136FDC
:1057E0000BB1506F9847230404D5054A936F0BB152
:1057F000D06F9847BDE81040FEF70EBF003C014057
:10580000A83F0020062108B50846FDF773FC0621D5
:105810000720FDF76FFC06210820FDF76BFC062131
:105820000920FDF767FC06210A20FDF763FC06212D
:105830001720FDF75FFCBDE8084006212820FDF792
:1058400059BC000008B5FFF743FE00F00DF8FDF766
:1058500067FCFDF777FEFDF74FFDFFF7F5FDBDE8AF
:105860000840FFF769BD00000023054A19460133CF
:10587000102BC2E9001102F10802F8D1704700BFF5
:10588000A83F002010B501390244904201D1002008
:1058900005E0037811F8014FA34201D0181B10BD99
:1058A0000130F2E72DE9F041A3B1C91A177801449C
:1058B000044603F1FF3C8C42204601D9002009E058
:1058C0000578BD4204F10104F5D10CEB0405D618AE
:1058D000A54201D1BDE8F08115F8018D16F801ED62
:1058E000F045F5D0E7E70000034611F8012B03F877
:1058F000012B002AF9D170476F72672E61726475AF
:1059000070696C6F742E663430355F4D6174656BF1
:10591000475053004E6F20617070207369670A0012
:10592000426164206677206C656E67746820257517
:105930000A0042616420626F6172645F69642025BD
:10594000752073686F756C642062652025750A0088
:105950004261642066772064657363726970746F56
:1059600072206C656E6774682025750A0042616458
:105970002061707020435243203078253038783AC7
:10598000307825303878203078253038783A3078BB
:10599000253038780A00476F6F64206669726D772A
:1059A0006172650A0040A2E4F1646891060000009B
:1059B00053544D3332463F3F3F00000053544D3364
:1059C00032463430780053544D3332463432780006
:1059D00053544D33324634343658580000000000DA
:1059E000B05900083F00000013040000BC59000833
:1059F0003F00000019040000C65900083F000000E5
:105A000021040000D05900083F0000000000000001
:105A100075320008613200089D32000889320008A2
:105A200095320008813200086D32000859320008B2
:105A3000A932000800000000010000000000000082
:105A40006D61696E0000000069646C650000000013
:105A5000485A000848360020C037002001000000E6
:105A6000C53B0008000000004172647550696C6F0E
:105A7000740025424F415244252D424C0025534588
:105A80005249414C250000000200000000000000C7
:105A900091340008FD34000840004000583C0020CC
:105AA000683C00200200000000000000030000002D
:105AB0000000000041350008000000001000000058
:105AC000783C002000000000010000000000000001
:105AD000303F002001010200B53F0008C53E00082C
:105AE000613F0008453F000843000000F05A0008ED
:105AF00009024300020100C0320904000001020251
:105B00000100052400100105240100010424020203
:105B10000524060001070582030800FF09040100AF
:105B2000020A00000007050102400000070581028B
:105B300040000000120000003C5B00081201100150
:105B40000200004009124157000201020301000057
:105B50000403090425424F41524425006634303580
:105B60002D4D6174656B47505300303132333435FD
:105B70003637383941424344454600000040000072
:105B80000040000000400000004000000000010054
:105B900000000200000002000000020000000200FD
:105BA00000000200000002000000020000000000EF
:105BB0007936000831390008DD390008400040001E
:105BC000903F0020903F002001000000A03F0020F7
:105BD000800000004001000003000000AA01A8129C
:105BE00000000000AAAAAAAA55011400FFBF0000E5
:105BF0008877000070A70A0000000A01000000007A
:105C0000AAAAAAAA00000001FFFF000000000000ED
:105C1000990000000000A01600000000AAAAAAA691
:105C200000005011FFDF00000000000000770800B6
:105C30002000000000000000AAAAAAAA100000008C
:105C4000FFFF00000008000000000000000000004E
:105C500000000000AAAAAAAA00000000FFFF00009E
:105C60000000000000000000000000000000000034
:105C7000AAAAAAAA00000000FFFF0000000000007E
:105C8000000000000000000000000000AAAAAAAA6C
:105C900000000000FFFF0000000000000000000006
:105CA00000000000000000000A00000000000000EA
:105CB00003000000000000000000000000000000E1
:105CC00000000000000000000000000000000000D4
:105CD000000000000000000038A5FF7F0100000068
:105CE000F60300000000000000000F0000000000AC
:105CF000640000000000000040420F00FE2A010086
:105D0000D2040000FF00960000000008009600008A
:105D10000000080004000000505B000800000000C4
:105D20000000000000000000000000000000000073
:045D3000000000006F
:00000001FF
